:1000000000400000C1000000ED000000F100000011
:10001000F5000000F9000000FD00000000000000F5
:1000200000000000000000000000000001010000CE
:100030000501000000000000090100000D010000A2
:100040001101000011010000110100001101000068
:100050001101000011010000110100001101000058
:100060001101000011010000110100001101000048
:100070001101000015010000190100001D01000020
:100080002101000025010000290100002D010000D0
:1000900031010000350100000000000000000000F8
:1000A000390100003D010000410100000000000096
:1000B00045010000490100004D0100005101000010
:1000C00000B583B0074B019304E0019B1A1D019218
:1000D00000221A60019A044B9A42F6D300F0B4F859
:1000E000FEE7C046D0020000D0020000FEE7C04696
:1000F000FEE7C046FEE7C046FEE7C046FEE7C04654
:10010000FEE7C046FEE7C046FEE7C046FEE7C04643
:10011000FEE7C046FEE7C046FEE7C046FEE7C04633
:10012000FEE7C046FEE7C046FEE7C046FEE7C04623
:10013000FEE7C046FEE7C046FEE7C046FEE7C04613
:10014000FEE7C046FEE7C046FEE7C046FEE7C04603
:10015000FEE7C04682B002006B4606331A80044BAD
:100160001B686A46063212881A80C04602B0704781
:10017000C0020000024B1B681B889BB2180070472E
:10018000C002000082B002006B4607331A70044BB5
:100190001B686A46073212781A70C04602B0704770
:1001A000C802000082B002006B4607331A70054B8C
:1001B0001B6801336A46073212781A70C04602B0D3
:1001C0007047C046C8020000024B1B681B889BB2E8
:1001D00018007047C4020000034B1B681B78DBB299
:1001E0009BB218007047C046CC020000034B1B684E
:1001F00001331B78DBB29BB218007047CC020000C1
:1002000000B583B00190019B002B01D1012307E0D1
:10021000019B013B1800FFF7F3FF0200019B5343D2
:10022000180003B000BDC04684B0019001230393C1
:1002300002E0039B01330393039A019B9A42F8DD8A
:10024000C04604B07047C04600B583B0194B1800D3
:10025000FFF780FF0DE0FFF7C9FF0300DBB21800D6
:10026000FFF790FFFFF7B8FF0300DBB21800FFF7BE
:1002700099FFFFF7A9FF03001A000F4B9A42EAD13A
:100280000E4B1800FFF766FFC046FFF79DFF031EE9
:10029000FBD1FFF7A1FF03001A00072313400193CE
:1002A000019B1800FFF7ACFF03009BB21800FFF79B
:1002B00051FFEEE7A5A50000FFFF000015A8000014
:1002C00000000050040000500000005004000050E6
:00000001FF
